:100000000C9420030C943D030C943D030C943D038D
:100010000C943D030C943D030C943D030C943D0360
:100020000C943D030C943D030C946B130C94AD1293
:100030000C94321B0C943D030C943D030C943D0333
:100040000C943D030C943D030C943D030C943D0330
:100050000C943D030C94E6140C943D030C943D0366
:100060000C943D030C943D030C943D030C943D0310
:100070000C943D030C943D030C943D030C943D0300
:100080000C943D030C943D030C943D030C943D03F0
:100090000C943D030C943D030C943D030C943D03E0
:1000A0000C943D030C943D030C943D03DD05510677
:1000B000E505AF05B305E905B605EC05F705C1058E
:1000C0004706C505FB05C905FF052906CD0503063D
:1000D0003306D30509061306BA05F005BD05F30579
:1000E000D8050E061F063F064106AB05E1055A0678
:1000F0008306890674067A068F0695069B064507D1
:10010000450778077807F207100818091809150835
:1001100089089A089A08590975097A097F09840992
:1001200089098E09930998099D09A209A909AC09B1
:10013000AF09B209B509B809BB09BE09C109C609A9
:10014000860D890DAE0DCE0DD60DE10DE40DE40D3D
:10015000E40DF00EF00E570E590E5E0E840EA70E33
:10016000AA0EAD0ED00EC510EC109512EC10951223
:1001700038115B119512501260120000000000004F
:10018000000000000000000000000000000000006F
:1001900000000000000000000000000000007E0FD2
:1001A00000D4FFFFFFC7000000780000000000003F
:1001B00000002A2B280000000000000000000000C2
:1001C000000000000029000000002C1E3420212225
:1001D00024342627252E362D3738271E1F2021228E
:1001E000232425263333362E37381F040506070807
:1001F000090A0B0C0D0E0F101112131415161718F7
:10020000191A1B1C1D2F3130232D35040506070834
:10021000090A0B0C0D0E0F101112131415161718D6
:10022000191A1B1C1D2F3130354C1E0F0500047F81
:100230003F1F643214643214783C1E1E140A0505F4
:10024000010902A10185020901A10005091901297D
:10025000081500250195087501810205010930097D
:10026000311581257F95027508810609381581258C
:100270007F950175088106050C0A38021581257FD6
:10028000950175088106C0C005010980A10185039B
:1002900019012AB700150126B700950175108100D4
:1002A000C0050C0901A101850419012AA00215014C
:1002B00026A002950175108100C00660FF0961A1AA
:1002C000010962150026FF00952075088102096367
:1002D000150026FF00952075089102C0050109064A
:1002E000A101050719E029E7150025019508750109
:1002F00081029501750881010507190029FF150084
:1003000026FF009506750881000508190129059545
:100310000575019102950175039101C009025B0009
:10032000030100A0FA0904000001030101000921F2
:1003300011010001224000070581030800010904A2
:100340000100020300000009211101000122220026
:1003500007058203200001070503032000010904AB
:1003600002000103000000092111010001227B00AD
:100370000705840320000112010002000000087537
:100380006F16550100010200011003730075007023
:1003900000650072003100360000001A033100755C
:1003A0000070006B006500790062006F00610072F0
:1003B000006400730000000403090422232526289A
:1003C000292A2C2D2F3032333536383A3B3D3E40EA
:1003D00042434547494A4C4E5051535557595A5C30
:1003E0005E6062646668696B6D6F71737577797B47
:1003F0007D7F81838587898A8C8E90929496989A46
:100400009C9E9FA1A3A5A7A8AAACAEAFB1B3B4B65A
:10041000B8B9BBBCBEBFC1C2C3C5C6C7C9CACBCCB5
:10042000CDCED0D1D2D2D3D4D5D6D7D7D8D9D9DA88
:10043000DADBDBDBDCDCDCDCDCDDDDDDDDDCDCDCFD
:10044000DCDCDBDBDBDADAD9D9D8D7D7D6D5D4D325
:10045000D2D2D1D0CECDCCCBCAC9C7C6C5C3C2C1FA
:10046000BFBEBCBBB9B8B6B4B3B1AFAEACAAA8A757
:10047000A5A3A19F9E9C9A98969492908E8C8A890F
:10048000878583817F7D7B79777573716F6D6B69EC
:1004900068666462605E5C5A5957555351504E4CC1
:1004A0004A4947454342403E3D3B3A383635333270
:1004B000302F2D2C2A29282625232224002500260A
:1004C00000250221002200230038001E001F00200A
:1004D000002D002700280037002152007C01000178
:1004E0000001000100010001000100010001000104
:1004F00000010001000100010001000100010001F4
:1005000000010001000100010001000100010001E3
:1005100000010001000100010001000100010001D3
:1005200000010001000100010001000100010001C3
:1005300000010001000100010001000001010101B2
:10054000010101010102020202020202020203038E
:10055000030303030303040404040404040505055E
:100560000505060606060607070707070808080820
:10057000090909090A0A0A0B0B0B0C0C0C0D0D0DCD
:100580000E0E0E0F0F0F1010111111121213131463
:1005900014151516161717181819191A1A1B1B1CDB
:1005A0001D1D1E1E1F202021222223242425262635
:1005B000272829292A2B2C2D2D2E2F30313232336A
:1005C0003435363738393A3B3C3D3E3F4041424373
:1005D0004445464748494A4C4D4E4F505153545557
:1005E0005658595A5B5D5E5F616264656668696B07
:1005F0006C6D6F7072737577787A7B7D7E80828385
:100600008587888A8C8E8F91939596989A9C9EA0C8
:10061000A2A3A5A7A9ABADAFB1B3B5B7BABCBEC0D5
:10062000C2C4C6C9CBCDCFD1D4D6D8DBDDDFE2E49E
:10063000E7E9EBEEF0F3F5F8FAFDFFFFAA7F55408E
:1006400011241FBECFEFDAE0DEBFCDBF11E0A0E086
:10065000B1E0E4E4FEE402C005900D92A239B107D6
:10066000D9F722E0A2E9B1E001C01D92A33CB20794
:10067000E1F70E94D1090C9420270C9400000E94FD
:10068000AA202FEF84E39CE0215080409040E1F7C6
:1006900000C000009AE088E10FB6F894A895809316
:1006A00060000FBE90936000FFCFA7E1B0E0EBE5E4
:1006B000F3E00C94DE264B8B5C8B6D8B7E8B8F8BEB
:1006C000611110920F0286E09E01235F3F4FD90116
:1006D000E82F1D92EA95E9F795E0FE017396D9019E
:1006E00001900D929A95E1F79C894E895F897B89EB
:1006F0007D879E876F87598B488BF901DE0117969E
:1007000001900D928A95E1F7CE0107960E94341967
:1007100081113EC086E0FE013796DE011196019000
:100720000D928A95E1F7FF81E8856A857B856115E1
:10073000710531F0EF3F31F481E0FF3F19F403C060
:1007400081E001C080E080FD23C02091D40130E031
:10075000C9010196877099274091050250E08417DE
:10076000950779F1F983EA837D836C8396E0929F04
:10077000D001939FB00D1124AB52BE4FFE013196B4
:1007800001900D929A95E1F78093D4010E94C118CF
:1007900016E0809105029091D4018917F9F0189F15
:1007A000C00111248B529E4F0E9434198823B1F04E
:1007B0008091050290E00196877099278093050249
:1007C000E8CF0E94AA201092D40110920502EEEC0C
:1007D000F1E086E0DF011D928A95E9F76796E3E094
:1007E0000C94FA26ADE0B0E0E8EFF3E00C94CF26ED
:1007F000FC018081918123813481232B31F09F3F43
:1008000031F491E08F3F19F403C091E001C090E012
:1008100090FDC3C57F0185E0DE01199601900D9220
:100820008A95E1F7F701228189859A85222349F08B
:100830000E94AF1F182F682F89859A850E941F205C
:1008400003C00E94EB1F182F69857A85812F0E94B3
:100850002A168C01F7018281882309F42BC19801A3
:10086000225037472031310508F040C18FEF93E027
:100870000E94D425811128C1025036EAA32EB12C42
:10088000002379F0A114F4E0BF0609F41DC1C501ED
:100890000E94D425811101C001502FEFA21AB20A83
:1008A000EFCFCE0101962C0188E0F20111928A95DA
:1008B000E9F72AE0322E85010F5F1F4FC5010E9424
:1008C000D42589831A82882309F4FEC0813009F077
:1008D00041C06501F2E0CF0ED11CC8010E94D425B1
:1008E0008A83882309F4F0C09FEF980F933060F457
:1008F00023E0A20EB11CC6010E94D4258B8388235D
:1009000009F4E2C01C8229C0843031F54E0133E085
:10091000830E911C02E010E056018FEFA81AB80A6E
:10092000C6010E94D425F40181934F01882309F464
:10093000CBC08C3741F4E2E0F0E0EC0FFD1FE00F9C
:10094000F11F10820AC00F5F1F4F650107301105AC
:1009500019F7BAC0580101C056018201F80120817F
:10096000222309F4A8CF213009F04CC081818130C5
:1009700049F46801F2E0CF0ED11CF80182810E9497
:10098000C3220AC0823051F46801F2E0CF0ED11CBC
:10099000F80182810E941E22860189C0833049F4B9
:1009A0006801F2E0CF0ED11CF80182810E94BA21C9
:1009B000F3CF843019F00F5F1F4F79C0F801228107
:1009C0000E5F1F4F80E090E030E0205331092A3065
:1009D000310568F4389EA001399E500D1124C901DB
:1009E000840F951F0F5F1F4FF8012081EDCF0097F7
:1009F00009F45DC0EFE9FFE03197F1F700C00000B6
:100A00000197F5CFE22FF0E0E655FE4F2490822FBC
:100A100086958695869590E0FC01E656FE4F64909B
:100A20002770712C022E02C0759467940A94E2F725
:100A3000F1E06F227724FC01E657FE4F8490912C61
:100A4000022E02C0959487940A94E2F731E0832243
:100A50009924FC01E658FE4FC490D12C02C0D594D5
:100A6000C7942A95E2F781E0C822DD24611471045D
:100A700019F081EE0E941E228114910419F086EE75
:100A80000E941E22822D0E94C3228114910419F01B
:100A900086EE0E94BA216114710419F081EE0E9461
:100AA000BA21C114D10419F08CE20E94C3220F5F55
:100AB0001F4F54CF011537E7130709F042C181E0FA
:100AC0000E9457200E94D60F80910602877009F479
:100AD00064C4F7018281882309F45FC480919A017C
:100AE00082FF5BC482E00E948D1857C40115F7E7AE
:100AF0001F0711F481E005C0013027E7120721F438
:100B000082E00E946420DECFF801E851FC47E73024
:100B1000F10508F4E5C0882309F45BC11092A8022E
:100B2000C8019057839708F013C184E090E00E94B9
:100B3000E22590939A0180939901F801E150F047E2
:100B4000E232F10520F4EA5AFF4F0C94B32680916B
:100B500099018160ACC080919A018860B4C0809195
:100B600099018260A4C08091990120C0809199016F
:100B700088609DC080919A011EC080919A01826018
:100B8000A2C080919901806192C080919901806298
:100B90008EC08091990180648AC00E94AA208091B1
:100BA0009901806884C080919901886084607FC0C9
:100BB00080919A018260816086C0809199018E7FC8
:100BC00076C080919A01877F7EC0809199018D7F48
:100BD0006EC08091990120C080919901877F67C084
:100BE00080919A011EC080919A018D7F6CC0809186
:100BF00099018F7E5CC0809199018F7D58C0809152
:100C000099018F7B54C00E94AA20809199018F770F
:100C10004EC080919901877F8B7F49C080919A0156
:100C20008D7F8E7F50C08091990182FB222720F911
:100C300091E0922790FB82F990FB83F938C0809174
:100C40009A01982F909591708E7F892B90FB81F956
:100C50003AC08091990186FB222720F991E09227E2
:100C600090FB86F924C00E94AA208091990187FBFD
:100C7000222720F991E0922790FB87F918C061E0C4
:100C800001C060E08EE090E00E94E8251EC08091E7
:100C9000990184FB222720F991E0922790FB84F9A7
:100CA00006C080919901982F909590FB80F98093D0
:100CB00099010BC080919A0183FB222720F991E0D2
:100CC000922790FB83F980939A016091990170912A
:100CD0009A0184E090E00E9406260E94AA20F4CEA9
:100CE000E858FF4F0C94B32606E221EE41EE6AE18C
:100CF0007CE705C007E225EE45EE6BE17CE7C70126
:100D00000E94D91BE1CE06E221EE40EE68E17CE7CD
:100D1000F6CF07E225EE44EE69E17CE7F0CF06E28C
:100D200021EE42EE6CE17CE7EACF07E225EE46EEEB
:100D30006DE17CE7E4CF08E221E045EE6EE17CE77F
:100D4000DECF013097E7190709F0DECE82E0B8CE9A
:100D50000631ECE71E0709F48AC203309CE7190745
:100D600021F140F40115FCE71F0789F001301C4711
:100D700011F13EC00B353CE7130739F10C358CE718
:100D80001807D9F00A351C4799F581E01FC00E9469
:100D9000AA20EFEFF4E32CE0E150F0402040E1F72F
:100DA00000C000000E94D5148FCE6FEF7FEF80E06F
:100DB00090E00E9406260E943F0380919A0182FBE8
:100DC000882780F991E0892701C080E00E94AA1855
:100DD0000FC00631FCE71F0709F459C280911002C9
:100DE0008272F801E052F847E531F10508F45DC27E
:100DF000F701828100811181882349F0C8010E9496
:100E0000AF1FD82E682FC8010E941F2004C0C80140
:100E10000E94EB1FD82EB8018D2D0E942A160E9429
:100E20003816B82E192F982EF7010281A580A294AA
:100E30009FE0A922809106028770B9F00023A9F0F3
:100E4000812F807F803421F080E28B0D883068F024
:100E500080919A0182FF09C082E00E948D188091E2
:100E600006028770DD24D3948111D12CC12EC29447
:100E70008FE0C8228C2D90E08C30910508F0D8C10D
:100E8000FC01E158FF4F0C94B326812F807F1F7027
:100E9000882311F01295107F0023B9F0112309F473
:100EA000B5C180E28B0D883010F0911006C0909192
:100EB0001002192B1093100205C090910F02192BEC
:100EC00010930F020E945118A1C18B2D0E94BA21CC
:100ED000112309F4ADC180E28B0D883088F199208F
:100EE00079F1109590910F02192310930F022BC0E6
:100EF000812F807F1F70803211F01295107F8B2D13
:100F0000992029F0F1E09F1609F441C04FC080916B
:100F10009A0182FD1BC0002369F0112339F09091E2
:100F20001002192B109310020E94511880E00E94A9
:100F30001E227EC180E00E94BA21112309F478C1EB
:100F4000812F0E944A180E94511872C1002381F01B
:100F500080911102AA2051F021E0A21207C0182BA3
:100F6000181709F465C11093110262C1812B16C0D4
:100F7000A11003C00E94441831C031E0A31609F447
:100F800057C1812F0E94D1200E94441851C10023D3
:100F900041F085E08A1508F44BC1812F0E94D820CA
:100FA00047C194E09A1508F443C118C0002349F0E2
:100FB000AA2099F3F701858180FF28C18F7085836E
:100FC000ECCFAA2059F0893309F02FC1FFEF27EEAB
:100FD00033E0F15020403040E1F725C1812F0E94DD
:100FE000D12026C1812F86958695837019F0813096
:100FF00061F01EC1002321F08B2D912F937002C050
:1010000080E090E00E94A71B19C1002321F08B2DE6
:10101000912F937002C080E090E00E94821B0EC16D
:10102000602F8B2D0E94E22009C1812F8370A9F5CA
:10103000011102C14B2D429546954770440F440F54
:101040008B2D8F7090E09C01042E01C0220F0A941A
:10105000EAF7B4FE08C08FE090E001C0880F4A951F
:10106000EAF7809501C080E016951695137012304E
:1010700069F088F490911202113019F0822B8923C3
:1010800002C0922B892B0E947020D6C0822B909197
:1010900012028927F8CF822BF6CF002319F0812F77
:1010A000817001C08695882309F4C6C04B2D4295F6
:1010B00046954770440F440F8B2D8F7090E09C0134
:1010C000042E01C0220F0A94EAF7B4FE08C08FE094
:1010D00090E001C0880F4A95EAF7809501C080E052
:1010E000169516951370123059F078F49091C50149
:1010F000113019F0822B892309C0922B892B06C04D
:10110000822B9091C501892701C0822B0E94542017
:1011100093C01F70002339F0812F0E9464208B2D13
:101120000E94D82089C08B2D0E94D120812F0E943F
:10113000572082C08B2D92EF991681F1991538F0C6
:10114000E0EF9E1659F0F1EF9F1619F15BC023EF07
:10115000921659F134EF9316C1F054C0002381F078
:1011600084E08A1508F464C01F7181E090E0012ECC
:1011700001C0880F0A94EAF79091C501892720C021
:1011800095E09A1508F454C0EFCF80919A0182FD42
:101190001AC0002329F0812F8F7127C00023D9F3B3
:1011A000812F8F710E94572043C0002341F01F718F
:1011B00081E0012E01C0880F0A94EAF701C080E0A7
:1011C0000E94542035C0002399F01F71812F0E9486
:1011D000642080919A0182FF07C0E8E01E9FC00151
:1011E0001124836080930602812F0E94642020C016
:1011F00081E00E948D18F1E0FA15D0F482E00E949F
:101200008D1816C0002321F0AA2029F28B2D8FCE35
:10121000AA2031F2893349F42FEF37EE83E02150D1
:1012200030408040E1F700C000008B2D0E94BA21C1
:1012300088EF8C0D843010F40E94CC1BDD2009F463
:10124000ACC08091060280FDA8C0F701128285958E
:10125000859585950E946420C7010E94F2038091C4
:1012600006028595859585950E94572096C08091A8
:1012700010028A7A91E009F490E090939401811130
:1012800012C069E286EC91E00E94681B09C080915F
:101290009401811180C069E286EC91E00E945B1BA1
:1012A0000E94511811CC65E3EDCFE557FF4F0C9428
:1012B000B3268091A10280FF12C08E7F8093A1028D
:1012C0006091A1027091A2028091A3029091A40268
:1012D0000E94062310921D020E945A1DF5CB8160C8
:1012E0008093A10261E086954EC047EF54E261E031
:1012F00075E22CC041E055E267EF74E227C04EE989
:1013000054E268EA74E222C048EA54E26EE974E208
:101310001DC044E854E261E974E218C041E954E2B6
:1013200064E874E213C04AE654E267E774E20EC070
:1013300047E754E26AE674E209C049E153E26BE22E
:1013400073E204C04BE253E269E173E20E943D1D87
:10135000BBCB61E081E017C065E082E019C068E0C6
:1013600086E016C06EE089E013C064E18FE010C033
:1013700067E185E10DC061E088E105C062E289E1D5
:1013800007C061E083E20E94B2249ECB6AE285E25C
:101390000E94291D99CB65E37FCF2D96E2E10C9445
:1013A000EB26AAE2B0E0E7EDF9E00C94CF2685B792
:1013B000806885BF85B7806885BF84B7877F84BF15
:1013C0000FB6F894A89580916000886180936000C2
:1013D000109260000FBE90E080E80FB6F894809302
:1013E0006100909361000FBE8BE195E190939301B2
:1013F000809392010E94F1120E9410138091E200EA
:1014000084608093E20078948091BB018823A1F0EE
:101410001091E9001F709091EC00892F817090FD70
:1014200080E8182B1092E9008091E80083FD0E946B
:10143000E20F1F701093E90082E084BD93E095BD38
:101440009AEF97BD80936E000E94101D811102C01B
:101450000E94001D0BE111E0EFE1EE2EE1E0FE2E17
:10146000D8018D918D018F3F11F00E946015E0161B
:10147000F106B1F70FE111E0F80181918F018F3F83
:1014800011F00E946015F1E003321F07A9F784E014
:10149000E6EAF1E0DF01282F1D922A95E9F7E5E958
:1014A000F1E0DF011D928A95E9F70E94D6178111BC
:1014B00002C00E94E21782E090E00E94D42580934F
:1014C000A00184E090E00E94E22590939A0180932D
:1014D00099010E947715EFE3FCE93197F1F700C01D
:1014E00000000E9477158091A60180FF08C06FEF71
:1014F0007FEF80E090E00E9406260E94D51483E0F2
:1015000090E00E94D4250E94702080919B0181115F
:1015100033C00E94D617811104C00E94E2170E94B6
:101520003D2388E090E00E94DC256093A102709347
:10153000A2028093A3029093A4026E7F71F40E9492
:101540003D2388E090E00E94DC256093A102709327
:10155000A2028093A3029093A4020E94F32210920D
:101560001D028091A10280FF04C060E086950E9468
:10157000B22481E080939B0184E091E09093AC02DF
:101580008093AB0268E1C62ED12C70E4572EBB24A9
:10159000B394AA24A3948E010F5F1F4F8091BB01C7
:1015A000853009F060C040E1E42E52E1F52E8091D3
:1015B000BB01853009F04AC08091BB01843009F439
:1015C00034C010921D0280919D0181110DC0A09226
:1015D0009D018091A102982F917090939C018E7F24
:1015E0008093A1020E945A1D1092AF020FB6F89488
:1015F000A895C09260000FBE5092600083B7817FB3
:10160000846083BF83B7816083BF7894889583B7F4
:101610008E7F83BF0FB6F894A89580916000886193
:1016200080936000109260000FBE8091BA01882301
:1016300009F4BDCF0E947715E6EAF1E081918111AE
:10164000D8C321E0EA3AF207C9F7B1CF0E94AA2035
:101650000E94CC1B10929D0180919C0181110E94DF
:10166000ED240E94441D0E94771521EAE22E21E01C
:10167000F22E36EA832E31E0932E25EA31E0D401B2
:10168000F70191918D9189272E173F0719F0882333
:10169000C1F322C0811120C00E94261B7C018091D1
:1016A0009E0190919F01E816F90609F447C08FEF5B
:1016B00089A38AA31BA20E94261B8160782F9DA369
:1016C0008CA349A15AA16BA18DA10E945503F09250
:1016D0009F01E0929E0132C0712CD4012D904D01EA
:1016E000F7013080322409F1612C44244394832D86
:1016F0008421A1F06EA27FA291E0822D842109F4C1
:1017000090E098A70E94261B8160782F9AA789A74E
:101710004EA15FA168A58AA50E9455036394440C5D
:10172000F4E06F12E4CFD7012C927394BFEFEB1A61
:10173000FB0AE4E07E12D1CF0E941A1B80911D02A9
:10174000882309F4AAC080911C02E091A102E695C9
:10175000E81BE0931802823059F4F0E0E55CFD4F9D
:10176000E491EE2EF12C96E0892E9BE1992E70C02B
:10177000863059F4F0E0E85CFD4FE491EE2EF12C58
:1017800086EF882E8AE1982E63C0893061F4E69551
:10179000F0E0EB5CFD4FE491EE2EF12CB5E88B2EE2
:1017A000BFE19B2E55C08F3061F4E695F0E0EE5C12
:1017B000FD4FE491EE2EF12CA7E28A2EAFE19A2E96
:1017C00047C0853159F4F0E0E15DFD4FE491EE2E24
:1017D000F12CF9ED8F2EFEE19F2E3AC08831F9F001
:1017E000833249F4EDE2F2E0E590F490ECEB8E2EDA
:1017F000EAE19E2E2DC08432D1F0853209F58E2F7C
:1018000063E00E947F26E92FF0E0E65DFD4FE49162
:10181000EE2EF12C70E9872E7DE1972E19C058E24B
:10182000E52EF12C6EE5862E6EE1962E11C034EF7A
:10183000E32EFF24F39446E2842E4EE1942E08C05A
:1018400090EDE92E97E0F92E2BEB822E2AE1922ED5
:1018500080911902882361F0109219020E94261BC0
:10186000909317028093160210921B0210921A0294
:101870000E94261BE0911602F09117028E1B9F0B0F
:101880008F3F9F4750F4EE0EFF1EF0921702E0923A
:10189000160286E192E0F401099586E0EDEBF2E0B4
:1018A000D80101900D928A95E1F71092BF02109233
:1018B000C0021092C1021092C2028B81811104C039
:1018C0008C81882309F451C08091BB029091BC02A5
:1018D0000E940C159C019091B602992309F4A7C2AD
:1018E0002531310508F441C09F3F19F09F5F909367
:1018F000B602FB80FF2061F00E9458251F1414F4EB
:1019000091E001C09FEF899F802D11248093BF0239
:10191000FC80FF2061F00E9458251F1414F491E010
:1019200001C09FEF899F802D11248093C0023091C8
:10193000BF023323D1F02091C0022223B1F045EB46
:101940003403C0011124992319F09093BF0202C0FF
:10195000B092BF0235EB2303C0011124992319F083
:101960009093C00202C0B092C0028D81811104C068
:101970008E81882309F451C08091B9029091BA02F6
:101980000E940C159C019091B702992309F454C24E
:101990002135310508F441C09F3F19F09F5F9093B6
:1019A000B702FD80FF2061F00E9436251F1414F459
:1019B00091E001C09FEF899F802D11248093C10287
:1019C000FE80FF2061F00E9436251F1414F491E080
:1019D00001C09FEF899F802D11248093C202309116
:1019E000C1023323D1F02091C2022223B1F045EB92
:1019F0003403C0011124992319F09093C10202C04D
:101A0000B092C10235EB2303C0011124992319F0D0
:101A10009093C20202C0B092C20246E050E0B80108
:101A20008DEB92E00E941327892BA9F48091BF02CD
:101A300081110FC08091C00281110BC08091C10241
:101A4000811107C081E09091C202911103C080E032
:101A500001C081E080FD0E940C2586E0F801ADEB1D
:101A6000B2E001900D928A95E1F70E94CC1B909113
:101A7000A501891721F08093A5010E941A1B80916E
:101A8000BB01843009F08ACD83E08093E900809126
:101A9000E80082FF83CD8091E80085FF21C00E948D
:101AA000421481111BC080E2E82EF12C480109C0CC
:101AB0008091F100D4018D934D01B1E0EB1AF10852
:101AC00069F08091E80085FDF3CF8091E8008B7785
:101AD0008093E8000E944214882399F391E001C0AA
:101AE00090E08091E8008B778093E800992309F4D7
:101AF00055CD2981822F90E0FC013197E331F1052A
:101B000008F06EC1E056FF4F0C94B3261A828BE0AA
:101B1000D3C08A81823009F482C150F4813009F047
:101B20005FC10E941A1B9B838C837D836E835AC185
:101B3000833041F0843009F053C11B821C821D8226
:101B40001E8250C18091A6018B838091A7018C8356
:101B50008091A8018D838091A90126C08A8182305D
:101B600019F0853051F03CC16B817C818D819E8163
:101B70000E94B9260E94DC1C35C18091A10280FF21
:101B80000AC08091A1028E7F8093A10210921D0253
:101B90000E945A1D27C10E94ED2424C14C816B81F3
:101BA0008A810E94AE1C9D838E831CC12D813E8143
:101BB0003227232732274C816B818A810E94521C55
:101BC00011C10E94791C0EC18A81823009F008C1BE
:101BD0002830B9F1293009F45FC08B818230F9F0E7
:101BE00098F4813009F0FEC08C81EFEF8E9FC00128
:101BF00011246FEF70E00E948B26462F20E0609149
:101C0000A3028091A2021AC08330A1F0843009F0AF
:101C1000E9C020E04091A4026D818C810FC08C81CD
:101C2000882309F4AECF0E94ED2460E08C810E94ED
:101C3000B224D8C08C818093A502D4C00E94F12325
:101C4000D1C08B818230E1F078F4813009F0CAC0D4
:101C50008091A402FFEF8F9FC00111246FEF70E00D
:101C60000E948B266C83BEC0833091F0843009F0D3
:101C7000B9C08091A2028C838091A3028D83B2C0EF
:101C80008091A10280FF02C0869504C080E002C05E
:101C90008091A5028C83A6C06091A1027091A202DE
:101CA0008091A3029091A4020E9406239BC080E130
:101CB00052C083E08A838AE58B8394C0EA80FB80EC
:101CC000FE24EF24FE248C80912C3801C7018A5514
:101CD0009F4F9301201B310B2815390508F082C056
:101CE0002AE5E21623E0F20630F40E94D425D3015F
:101CF00014968C9302C0F3011482FFEFEF1AFF0ACF
:101D00002FEF621A720AE2CFEA80FB80FE24EF24F2
:101D1000FE248C80912C3801C7018A559F4F930176
:101D2000201B310B2815390508F05CC03AE5E31695
:101D300033E0F30628F4D30114966C910E94E82551
:101D4000BFEFEB1AFB0AEFEF6E1A7E0AE5CF0E9497
:101D5000421C48C084E08A8345C0EA80FB80FE24A0
:101D6000EF24FE248C80912C3801C70186969301C4
:101D7000201B310B28153905A8F5F0E8EF16F10402
:101D800030F40E94D425D30114968C9302C0F30141
:101D90001482FFEFEF1AFF0A2FEF621A720AE5CFE3
:101DA000EA80FB80FE24EF24FE248C80912C3801F5
:101DB000C70186969301201B310B2815390590F435
:101DC00030E8E316F10428F4D30114966C910E94D4
:101DD000E825BFEFEB1AFB0AEFEF6E1A7E0AE8CF99
:101DE0008FEF898340E250E0B80182E00E947514D1
:101DF000D5CBE9BCF9BC09B400FEFDCF8091D80079
:101E00008F7D8093D8008091E00082608093E00015
:101E10008091E00081FDFCCF0E94AA20C8CB85E222
:101E200090E00E94D4251B821C821D82BDCE2B30E7
:101E3000310508F05BCD99CD2B30310508F0AECDE2
:101E4000ECCD8091BD0187FF11C08091E80082FD3B
:101E500005C08091BB018111F8CF11C08091E800CD
:101E60008B770BC08091BB01882349F08091E800FB
:101E700080FFF8CF8091E8008E778093E800089586
:101E8000982F973068F59093E900981739F0709182
:101E9000EC002091ED005091F00003C0242F762F2C
:101EA00050E021FD02C09F5FECCF3091EB003E7F00
:101EB0003093EB003091ED003D7F3093ED00309199
:101EC000EB0031603093EB007093EC002093ED0059
:101ED0005093F0002091EE0027FDE5CF80E00895BB
:101EE0008F708093E90081E008952091C3013091C3
:101EF000C4012617370748F06115710539F42091A0
:101F0000E8002E772093E80001C0B901FC0120E031
:101F10006115710579F18091BB018823F1F185305C
:101F2000F1F18091E80083FD3CC08091E80082FDE2
:101F30002EC08091E80080FFEBCF2091F3008091CC
:101F4000F20090E0922B6115710551F088309105F7
:101F500038F421912093F100615071090196F3CF7B
:101F600021E0089709F020E08091E8008E778093C7
:101F7000E800CECF2111CFCF0AC08091BB018823CA
:101F800061F0853061F08091E80083FD0AC08091A6
:101F9000E80082FFF2CF80E0089582E0089583E0B8
:101FA000089581E008958091B00108958091C50160
:101FB000982F9670963011F4886001C0877F0E9438
:101FC00054200895AAE2B0E0E8EEFFE00C94DE268B
:101FD000EDEBF1E085EC91E02091F10021938E177B
:101FE0009F07D1F78091BE01833009F463C030F4BC
:101FF000813071F0823009F49DC0B4C08A3009F498
:1020000089C08B3009F46EC0893009F0ABC020C0A4
:102010008091BD01813A09F0A5C08091E800877FD9
:102020008093E8008091C1019091C201892B21F435
:1020300068E081EB91E003C060E080E090E070E058
:102040000E94750F8091E8008B778093E8008AC02A
:102050008091BD01813209F085C08091C1019091CC
:10206000C201009719F0029709F07CC08091E80046
:10207000877F8093E8008091E80082FD05C0809111
:10208000BB018111F8CF6EC02091F3008091F20066
:1020900090E0922B029731F48091F100813011F0A1
:1020A000863021F48091F1008093B0018091E800A6
:1020B0008B7754C08091BD01813A09F053C0809163
:1020C000C1019091C201892B09F04CC08091E800B8
:1020D000877F8093E8008091E80080FFFCCF8091AB
:1020E0000C0137C08091BD018132E1F58091C101C1
:1020F0009091C201892BB1F58091E800877F809390
:10210000E8000E94210F8091BF0180930C010E9482
:10211000AA2028C08091BD01813221F58091E8007C
:10212000877F8093E8000E94210F8091C0018093F7
:10213000AF0118C08091BD01813AA1F48091E800FF
:10214000877F8093E8008091E80080FFFCCF80913A
:10215000AF018093F1008091E8008E778093E800D2
:102160000E94210F8091E80083FFDFC18091BD01B3
:102170009091BE01492F50E04A30510508F0D5C179
:10218000FA01ED54FF4F0C94B326803821F08238C9
:1021900009F0CBC108C08091B9019091BA0199238F
:1021A00089F082600FC08091C1018F70873008F084
:1021B000BCC18093E9008091EB0085FB882780F902
:1021C0001092E9009091E800977F9093E800809347
:1021D000F1001092F10070C1282F2D7F09F0A5C1E8
:1021E000882319F0823061F0A0C18091BF01813055
:1021F00009F09BC1933009F080E08093BA012EC0B2
:102200008091BF0181112AC08091C1018F702FEF91
:10221000280F263008F089C18093E9002091EB0057
:1022200020FF1CC0933021F48091EB00806214C029
:102230009091EB0090619093EB0021E030E0A901D8
:1022400002C0440F551F8A95E2F74093EA001092AE
:10225000EA008091EB0088608093EB001092E90027
:102260008091E800877F8093E8000E94210F5DC184
:1022700081115BC11091BF011F778091E3008078CD
:10228000812B8093E3008091E800877F8093E800B2
:102290000E94210F8091E80080FFFCCF8091E30035
:1022A00080688093E300111102C082E001C083E0E6
:1022B0008093BB013AC18058823008F036C120912A
:1022C000BF013091C0012C3D53E0350779F583E023
:1022D0008A838AE289834FB7F894DE01139620E05F
:1022E0003EE051E2E32FF0E050935700E49120FFED
:1022F00003C0E295EF703F5FEF708E2F90E0EA3001
:1023000010F0C79601C0C0968D939D932F5F243126
:1023100049F74FBF8091E800877F8093E8006AE229
:1023200070E0CE0101960E94750FB4C08091C1018A
:102330009091C201432F552743305105A9F068F40D
:102340004130510509F400C14230510509F0EDC09A
:102350008BE590E0ECE1F3E04BC04132510529F10F
:102360004232510589F1E1C0C901992781309105B7
:10237000A1F058F0029709F0D8C0E9E8F3E0E49141
:102380008E2F90E0E9E8F3E030C0E7EBF3E0E49172
:102390008E2F90E0E7EBF3E028C0EBE9F3E0E49167
:1023A0008E2F90E0EBE9F3E020C08330910508F038
:1023B000BCC0880F991FFC01E45DFE4F0190F081C5
:1023C000E02D89E090E014C08330910508F0ADC0A5
:1023D000FC01EE0FFF1FEA5DFE4F0190F081E02D42
:1023E000DC01AD5DBE4F8C9190E0009709F49DC07B
:1023F0002091E800277F2093E8002091C3013091CD
:10240000C4012817390708F4C90140E0009789F191
:102410002091BB01222309F43DC02530D9F1209140
:10242000E80023FD37C02091E80022FD2FC0209155
:10243000E80020FFEBCF4091F3002091F20030E064
:10244000342B009759F02830310540F444914093E3
:10245000F100319601972F5F3F4FF3CF41E02830D5
:10246000310509F040E02091E8002E772093E80044
:10247000CDCF4111CDCF0AC08091BB01882351F04F
:10248000853041F08091E80083FD04C08091E80030
:1024900082FFF2CF8091E8008B778093E80045C0FF
:1024A000803809F042C08091E800877F8093E8007F
:1024B0008091BC018093F1008091E8008E77D3CEAB
:1024C000811133C08091BF019091C001992702977B
:1024D00064F58091E800877F8093E8001091BF0148
:1024E0001093BC010E94210F111106C08091E300DE
:1024F00087FD02C081E001C084E08093BB0142E01F
:1025000061EC81E00E94400F42E261EC84E00E94B5
:10251000400F42E261EC82E00E94400F42E260EC38
:1025200083E00E94400F8091BB018091E80083FF0F
:1025300010C08091E800877F8093E8008091EB00D5
:1025400080628093EB0005C082E190E0E7E7F3E072
:102550004FCFAA96E3E00C94FA261F920F920FB683
:102560000F9211242F933F934F935F936F937F9319
:102570008F939F93AF93BF93CF93DF93EF93FF938B
:10258000C091E900CF708091EC00D82FD17080FD10
:10259000D0E81092E9008091F000877F8093F000EE
:1025A00078940E94E20F1092E9008091F000886018
:1025B0008093F000CD2BCF70C093E900FF91EF9195
:1025C000DF91CF91BF91AF919F918F917F916F914B
:1025D0005F914F913F912F910F900FBE0F901F90E1
:1025E0001895E8EDF0E080818E7F80831092E20004
:1025F0001092DA001092E100A0EEB0E08C918160C0
:102600008C9380818F77808319BCA7EDB0E08C918B
:102610008E7F8C9380818F7E80831092AE0108958F
:10262000A0E0B0E0E6E1F3E10C94D926C8EDD0E0FB
:1026300088818F7E8883E7EDF0E0808181608083F0
:1026400084E082BF81E08093AE0188818E7F8883A1
:1026500002EE10E0F80110821092DA0081EEC82E2E
:10266000D12CF601108288818F77888388818068D9
:10267000888388818F7D888319BC1092BB0110925A
:10268000BC011092BA011092B90190EEE92EF12C22
:10269000F70180818B7F808388818160888342E01D
:1026A00060E080E00E94400FF60180818E7F808391
:1026B000F801808181608083808188608083F70158
:1026C00080818E7F8083888180618883CDB7DEB7EB
:1026D000E8E00C94F5261F920F920FB60F9211248A
:1026E0002F933F934F935F936F937F938F939F931A
:1026F000AF93BF93EF93FF938091E10082FF09C0F6
:102700008091E20082FF05C08091E1008B7F809381
:10271000E1008091DA0080FF2AC08091D80080FF1C
:1027200026C08091DA008E7F8093DA008091D900F4
:1027300080FF18C080E189BD82E189BD09B400FE37
:10274000FDCF81E08093BB018091AE0181110FC06C
:102750000E94F1120E9410138091E2008460809325
:10276000E20005C019BC1092BB011092AE0180912D
:10277000E10080FF17C08091E20080FF13C08091CC
:10278000E2008E7F8093E2008091E200806180937E
:10279000E2008091D80080628093D80019BC85E067
:1027A0008093BB018091E10084FF30C08091E20002
:1027B00084FF2CC080E189BD82E189BD09B400FE9F
:1027C000FDCF8091D8008F7D8093D8008091E1006B
:1027D0008F7E8093E1008091E2008F7E8093E20003
:1027E0008091E20081608093E2008091BC018823A7
:1027F00011F084E007C08091E30087FD02C081E012
:1028000001C083E08093BB018091BB018091E10016
:1028100083FF27C08091E20083FF23C08091E10005
:10282000877F8093E10082E08093BB011092BC011E
:102830008091E1008E7F8093E1008091E2008E7FA5
:102840008093E2008091E20080618093E20042E0A8
:1028500060E080E00E94400F8091F00088608093EB
:10286000F000FF91EF91BF91AF919F918F917F9178
:102870006F915F914F913F912F910F900FBE0F90ED
:102880001F9018952091E4003091E50095E6409165
:10289000EC00842F817040FF23C08091E80080FD10
:1028A0001DC08091BB01882399F0853099F08091FB
:1028B000EB0085FD11C04091E4005091E500241724
:1028C000350729F3915011F09A01E1CF84E0089582
:1028D00082E0089583E0089581E0089580E00895FE
:1028E0004091E80042FFDDCF08950F931F93CF93EF
:1028F000DF938B01EA019091BB01943079F58F70E1
:102900008093E9008FEF9091E800815095FD06C01B
:1029100095ED9A95F1F700008111F5CF8091E800CF
:1029200085FF1CC00E944214882361F08091E8005A
:102930008E778093E80012C0F80181918F01809317
:10294000F1002197209791F38091E80085FDF4CF65
:102950008091E8008E778093E800E4CFDF91CF91FB
:102960001F910F91089543E050E0BC0184E00E9464
:102970007514089546E050E0BC0184E00E9475148F
:102980000895CF93DF93EC0148E050E0BC0181E073
:102990000E94751488E0FE01A1EBB1E001900D9258
:1029A0008A95E1F7DF91CF91089587E797E79093B4
:1029B0000108809300089AE088E10FB6F894A89582
:1029C000809360000FBE90936000FFCF78941F92B9
:1029D0000F920FB60F9211248F939F93AF93BF93D3
:1029E0008091AA019091AB01A091AC01B091AD0191
:1029F0000196A11DB11D8093AA019093AB01A093F4
:102A0000AC01B093AD01BF91AF919F918F910F90A9
:102A10000FBE0F901F9018959C014FB7F8948091AE
:102A2000AA019091AB01A091AC01B091AD014FBF53
:102A3000821B930B089580E008959091990192FF75
:102A40000DC0282F2871283019F4877F846006C0B4
:102A5000282F2471243011F48B7F886093FF0DC0E0
:102A6000282F2871283119F4877E846106C0282F09
:102A70002471243111F48B7E886120919A0120FF0A
:102A80000DC0382F3871383019F4877F816006C047
:102A9000382F3171313011F48E7F886021FF0DC0E5
:102AA000282F2871283119F4877E816106C0282FCC
:102AB0002171213111F48E7E886194FD877E089505
:102AC000F894E82FE295EF70F0E031A1282F2F70F5
:102AD00081E090E001C0880F2A95EAF7982F909541
:102AE000932391A392A1892B82A378940895A4E0C3
:102AF000B0E0EDE7F5E10C94D62619821A821B822C
:102B00001C820BE111E0AE014F5F5F4F7A015A0169
:102B1000CC24C394D12CF80180818F3F09F441C0AB
:102B2000F894E82FE295EF70F0E021A18F70A601F4
:102B300002C0440F551F8A95E2F7CA01922F982BC5
:102B400091A392A18095892382A3789400C0EFE19C
:102B5000F1E0912C31E021912F3F89F0A22FA29535
:102B6000AF70B0E090968C9190E02F7002C0959578
:102B700087952A95E2F780FD02C0832F01C080E08F
:102B8000982A330F51E0E332F50729F7F8018081E5
:102B90008F3F11F00E946015F0EAFA95F1F7F70106
:102BA00090820F5F1F4FFFEFEF1AFF0A41E00F31D6
:102BB000140709F0B0CF44E050E0B50185E991E099
:102BC0000E941327892BA9F089819A81AB81BC814E
:102BD0008093950190939601A0939701B0939801EB
:102BE00081E0809315020E94261B9093140280932B
:102BF000130280911502811102C080E027C08091EC
:102C00001302909114020E940C150597B0F344E052
:102C100050E065E971E086EA91E00E941327892B74
:102C200091F08091950190919601A0919701B091BA
:102C300098018093A6019093A701A093A801B09357
:102C4000A90181E001C080E0109215022496EBE01A
:102C50000C94F226743048F4643038F4843028F44C
:102C6000462F672F0E94AE1C089580E090E00895E3
:102C7000CF93DF938238910569F1B0F481339105E8
:102C800009F477C048F48932910509F469C08A32A1
:102C9000910509F473C092C08533910509F45BC0B6
:102CA00089339105B9F08AC0833E910591F138F4DA
:102CB000803E9105D1F0823E910531F17FC0863E84
:102CC0009105D9F1873E9105E9F1843E910509F01E
:102CD00075C028C02091990120FD5BC021FD59C01D
:102CE00020919A0123FD61C069C08091990180FD06
:102CF0004AC080919A0180FF4CC08091990184FD67
:102D000050C183EE90E04FC18091990182FF3EC097
:102D1000F4CF8091990182FD39C080919A0180FDA4
:102D200038C0EBCF80919A0181FF39C08091990121
:102D300084FD37C187EE90E036C18091990183FF11
:102D40002BC0F4CF8091990183FD26C080919A0118
:102D500081FD25C0EBCF8091990185FD26C022C061
:102D60008091990185FD1EC080919A0183FF1DC04D
:102D70000AC08091990186FD1BC01DC080919901F8
:102D800086FD19C015C089E390E00DC182EE90E088
:102D90000AC180EE90E007C186EE90E004C184EEA7
:102DA00090E001C185E390E0FEC089E290E0FBC0C5
:102DB0008AE290E0F8C081E390E0F5C0EC01811573
:102DC00030E5930708F053C0811560E4960720F0C2
:102DD000CE019F70906AE7C0803E910588F58D3CDA
:102DE000910518F0CE019065DEC0883A9105C0F4D7
:102DF000853A910550F08C2F855AC82FD0E0CE5CD3
:102E0000DE4F888190E09064CEC08130910509F456
:102E1000C5C008F4C6C0049708F4C3C0CE01C3C03F
:102E2000813C910508F0BDC08C2F885AC82FD0E096
:102E3000CC0FDD1FCB5CDE4F888199819464B3C0D9
:102E40008115904258F08D2F8F710E941D15282FEB
:102E50002F71CE0199279062922BA5C0C11581E0F8
:102E6000D807E0F6C83ED10508F09BC0D7CFC036E2
:102E700092E5D90708F053C0C03422E5D207B8F074
:102E80008C2F8F718695869570E2879FA001112403
:102E90008C2F837021E030E0B90102C0660F771FEC
:102EA0008A95E2F7CB019C68842B952B7CC0C032BD
:102EB00032E5D30740F08C2F8F7190E0982F882750
:102EC000816F906A70C0C11562E5D607B0F08C2F93
:102ED0008695869520E2829FA00111248C2F837015
:102EE00021E030E0B90102C0660F771F8A95E2F752
:102EF000CB01842B952B9D6856C08C2F8F710E941F
:102F00001D1595E0D695C7959A95E1F7CF70D0E05D
:102F1000DC2FCC27D0699E01282BC90144C0C03AC0
:102F200072E5D70708F58C2F8F71C03892E5D90765
:102F3000A8F48695869570E2879F900111248C2FC6
:102F4000837041E050E0BA0102C0660F771F8A9596
:102F5000E2F7CB019A68822B932B25C090E0982F43
:102F60008827846F906A1FC0C03C22E5D20750F4C6
:102F70008C2F8F710E941D158F7190E0982F8827DC
:102F8000906211C0C03E32E5D30758F4CE018F7174
:102F90009927982F8827806F906A05C081E090E07C
:102FA00002C080E090E0DF91CF91089580E090E052
:102FB0000E94E225873E9E4F19F40E94101D08953D
:102FC00080E0089567EE7EEF80E090E00E940626A4
:102FD00060E082E090E00E94E82560E083E090E01D
:102FE0000E94E8251092120260E074E184E090E013
:102FF0000E94062660E086E090E00E94E8256FEFE0
:1030000087E090E00E94E82540E050E0BA0188E0C7
:1030100090E00E94FA2560E08DE090E00E94E825B3
:1030200040E050E0BA0188E190E00E94FA2560E0BB
:1030300087E190E00E94E82540E050E0BA018CE191
:1030400090E00E94FA2560E070E080E290E00E944B
:10305000062640E050E0BA0188E190E00E94FA259F
:1030600080E00E94E11C0E94001D40E050E0BA0197
:103070008FE090E00E94FA2540E050E0BA0183E141
:1030800090E00E94FA25089580911102811110921A
:103090001102089580959091100289238093100267
:1030A00008959091100280910F02982B9093C60181
:1030B00080911102882389F0892B8093C601E8EC66
:1030C000F1E097E080E0915029F021912223D9F39B
:1030D0008F5FF9CF81110E94441848E050E067E00B
:1030E00072E086EC91E00E941327892BA9F088E01A
:1030F000E6ECF1E0A7E0B2E001900D928A95E1F7ED
:10310000E091AB02F091AC02309731F00280F38194
:10311000E02D86EC91E009950895209106028095B6
:10312000822380930602982F977099F430E0482FFD
:10313000082E000C550B2417350759F090919A0171
:1031400092FF07C08595859585950E94572010921E
:103150000602089590919A0192FB222720F92817E0
:1031600079F080FB92F990939A01609199017091A6
:103170009A0184E090E00E94062682E00E948D1869
:103180000895809105029091D401891719F08F5FFD
:103190008770FBCF08950F931F93CF93DF93809198
:1031A000D30182958F7009F05AC08091D001882395
:1031B00009F455C0809105021091D4016091CE01AF
:1031C0007091CF01C091D101D091D20191E06F3FB8
:1031D00009F090E0292F06E0811709F440C02097FC
:1031E00021F07F3F21F030E003C031E001C0322FF9
:1031F00090E030FD31C0089FF001099FF00D1124CF
:10320000DF01AB52BE4F11963C911197371324C08A
:103210003C91361321C012963C91129731111CC07B
:1032200013964D915C9114974C1B5D0B483C5105D6
:1032300098F48091D3018F7080618093D301E6521E
:10324000FE4F80818F70806180838EEC91E00E94C0
:10325000F2030E94C11803C001968770BDCFDF91B1
:10326000CF911F910F910895A1E1B0E0EAE3F9E158
:103270000C94D6268C0185E0F801DE011D960190A4
:103280000D928A95E1F7F801E2809091CE0160916C
:10329000CF014091D1015091D2014115510531F03A
:1032A0006F3F31F481E09F3F19F403C081E001C01A
:1032B00080E0F82FF1709F2E80FD1BC1F801308156
:1032C0002181C380D4808EECA82E81E0B82EF090AE
:1032D000D001F601E41BF50BFF2009F4C7C0809173
:1032E000D301E83CF10508F092C0482F407F09F077
:1032F00051C0621311C093130FC0FE2CE1100CC01B
:103300008F7080618093D301C5010E94F203809188
:10331000D301F80185832AC1C114D10431F02F3FB4
:1033200031F481E03F3F19F403C081E001C080E047
:1033300080FD03C081E08E2502C080E090E0F82F80
:10334000F170FF2E80FF1CC0809105024091D401D6
:1033500056E0841709F4E8C090E0589FF001599FA7
:10336000F00D1124EB52FE4F6181261306C06081DF
:10337000631303C06281E61203C001968770E9CF30
:10338000FE2CEE2009F4F2C08091D301816080937D
:10339000D30149C0621306C0931304C0E11002C0F8
:1033A000F80186C0C8010E947320882351F1EE20E5
:1033B00041F12091D301822F82958F7090E0029786
:1033C00074F08091CE019091CF0198878F831986F8
:1033D000DB86CA862C87CE0107960E94F20386E020
:1033E000F801AEECB1E001900D928A95E1F70E94F0
:1033F000CB180AC06217C9F0C8010E94732081115E
:103400001EC0C8010E94F203FF24F394AFC0482FEE
:10341000407F81F78EEC91E00E94F20386E0F50197
:1034200011928A95E9F7F12CA1C09313E5CFE11031
:10343000E3CFF8018583C8010E94F20354C0EE2057
:1034400001F32091D301822F82958F7090E0029733
:1034500034F28091CE019091CF019A8389831B82AF
:10346000DD82CC822E83CE010196B7CFE83CF105F8
:10347000D0F5FE2CEE2029F2621327C0931325C04D
:103480002091D30120FD18C0822F82958F70482F84
:1034900050E04115510581F0F80125834F30510569
:1034A00041F08F5F982F9295907F822F8F70892B9C
:1034B0008583C8010E94F20386E0F801AEECB1E01A
:1034C00001900D928A95E1F751C0C8010E947320C6
:1034D000811185CF8091D30181608093D301C80190
:1034E0000E94F20343C086E0F50111928A95E9F744
:1034F0003DC0EE2009F485CFC8010E947320F82E4C
:10350000882309F47ECF86E0F801AEECB1E00190AB
:103510000D928A95E1F78091CE019091CF010E94A2
:10352000DE1F0E94CB1822C03D872E878D859E8589
:103530000E94DE1F292F22952F70223028F49F70C1
:1035400039F0811105C00BC0243028F49F7049F474
:10355000805E883020F0C8010E94F2039F2CF92C75
:1035600005C0F8019581907F99F7F9CF8F2D61966D
:10357000EBE00C94F2260895A3E0B0E0E2ECFAE16F
:103580000C94DD268C018091200281110AC09E01DD
:103590002F5F3F4F4FEF6FEF0E944D238A81809343
:1035A0002002F8018481813051F028F0823061F4EA
:1035B000409120020AC08091200240E007C0609143
:1035C000200240E080E003C040E080E060E00E9434
:1035D000E222F801848190E0019663E070E00E94AD
:1035E0009F2684832396E4E00C94F926CF93DF93FF
:1035F000EC01E1EAF2E0438162818C810E94D923EF
:103600008C818F5F8C83DF91CF910895CF93DF936F
:10361000EC01EC81F0E0E554FC4F4491E1EAF2E08A
:10362000628181810E94D9238C818F5F8C83DF919D
:10363000CF9108952FB7F8946091AA017091AB01D2
:103640008091AC019091AD012FBF08952FB7F894F0
:103650008091AA019091AB01A091AC01B091AD0114
:103660002FBF08951F920F920FB60F9211248F93C0
:103670009F93AF93BF938091AF02811113C080914C
:10368000AA019091AB01A091AC01B091AD0141961E
:10369000A11DB11D8093AA019093AB01A093AC0131
:1036A000B093AD01BF91AF919F918F910F900FBEDD
:1036B0000F901F9018959C012A5F3F4FFC0142819B
:1036C000461301C01282019682179307B9F7089535
:1036D0009C01FC0132969FEF80E04191461789F0F2
:1036E0009F3F19F4411101C0982F8F5F8630A9F7D1
:1036F0009F3F39F0F901E90FF11D97FDFA956283BB
:1037000008950895A3E0B0E0E8E8FBE10C94DF261B
:103710002091AD023091AE0228173907A1F09093A5
:10372000AE028093AD02E091AB02F091AC02309713
:1037300051F024E029839B838A830680F781E02D62
:10374000CE01019609952396E2E00C94FB26A3E0B6
:10375000B0E0EDEAFBE10C94DF262091A902309164
:10376000AA0228173907A1F09093AA028093A90210
:10377000E091AB02F091AC02309751F023E0298345
:103780009B838A830680F781E02DCE0101960995FF
:103790002396E2E00C94FB26E091AB02F091AC02A0
:1037A000309729F00190F081E02D0995089580E08F
:1037B00008950F931F93CF93DF93C42FD22FFC0153
:1037C00082818823B1F04093A8020E94261B909327
:1037D000A7028093A60280E28C0F883008F04DC0CB
:1037E000C77081E001C0880FCA95EAF70E94D8200F
:1037F00044C08091A802481330C08091A6029091E5
:10380000A7020E940C15883C910538F510E21D0FA7
:10381000CD17B9F080E28C0F883040F4C77081E09A
:1038200001C0880FCA95EAF70E94D120183010F520
:1038300081E09D2F977001C0880F9A95EAF70E944A
:10384000D820802F0E94C3221830B8F4D77081E0AE
:1038500001C0880FDA95EAF70AC080E28C0F883041
:1038600060F4C77081E001C0880FCA95EAF70E9432
:10387000D12003C0802F0E94C322DF91CF911F91DE
:103880000F910895CF93DF93C6EAD0E060E0CE01B8
:103890000E94E8252196C11584E0D807B9F7DF9189
:1038A000CF9108951F93CF93DF93962F8430E8F440
:1038B0006430D8F44430C8F4632F122FC42FD0E002
:1038C000CC0FDD1F28E0929FC00DD11D112490E286
:1038D000899FC00DD11D1124CE0186960E94E82536
:1038E000612FCE0187960E94E825DF91CF911F912D
:1038F0000895A0E0B0E0EFE7FCE10C94D726A12CFE
:10390000E12CF12CB12C00E010E0C0E0D0E0670128
:10391000C00ED11EF601EC0FFD1FEE0FFF1FE55488
:10392000FB4F259134914C2F6B2D8A2D0E94521CF8
:103930002196C430D10571F70C5F1F4FB39484E01A
:10394000B812E3CF80E1E80EF11CA39484E0A81242
:10395000D9CFCDB7DEB7EAE00C94F3260F931F93CF
:10396000CF93DF93843008F56430F8F44430E8F402
:10397000C42FD0E0CC0FDD1F28E0629FC00DD11D09
:10398000112430E2839FC00DD11D1124CE018696F3
:103990000E94D42590E0182F0027CE0187960E9420
:1039A000D4259801282BC90102C080E090E0DF9166
:1039B000CF911F910F91089585E290E00E94E82534
:1039C0000895CF93C82F811102C06FEF01C062E24A
:1039D00082E290E00E94E825C11102C06FEF01C0B1
:1039E00062E183E290E00E94E825C11102C06FEF1E
:1039F00001C068E084E290E00E94E825CF9108953C
:103A000080E00E94E11C60E070E0CB010E94DC1CC1
:103A10000E94791C0E94421C81E00E94E11C0895D2
:103A200082E290E00E94D425823281F483E290E029
:103A30000E94D425823151F484E290E00E94D42582
:103A400091E0883009F090E0892F01C080E081701A
:103A500008959091A10290FF04C09695981748F0A0
:103A600003C0811106C090E0961718F40E9401254A
:103A7000089561E00E94B2240895882311F0FA01AC
:103A800001C0FB01099508956091A102669570E05F
:103A90004BE050E08DE091E00E940627892B19F45D
:103AA00081E080931D020E94261B90931702809351
:103AB000160208958091A10280FF0AC0539A8BB12B
:103AC000877F9BB198602FB7F894E1E2F2E00BC0DA
:103AD000E1E2F2E0118210821282339632E0E135A7
:103AE000F307C1F7EBCF32E0E135F30789F031910D
:103AF00048E09BB9000000C037FF8BB9330F0000CE
:103B000000C000C000C08BB900C04A9591F7EBCF50
:103B10002FBF8FE594E00197F1F700C000000895F2
:103B2000A0E0B0E0E6E9FDE10C94D626FC01A2801D
:103B3000948081E08483EBEBF3E0B490EAE3F4E07B
:103B4000E491C1E5D2E0F1E2EF2EF2E0FF2ECC24C9
:103B5000CA94D12CEB190E2F10E022E02A1530F078
:103B60008091A20288838091A3028983911003C06F
:103B70001B821A8255C08B818823F9F081508B8378
:103B80002FEF829FC00111246C8170E00E948B2670
:103B9000FB01FF27E554FC4F8491E82FEB192FEF31
:103BA000E29FC0011124B8010E948B268091A402DB
:103BB000689FB00111247A8333C00E94C4252091EC
:103BC000A4022695215830E0A901440F551F322F39
:103BD0002227240F351F232F33278217930704F53D
:103BE00082E08A1588F40E94C425B6010E949F26AF
:103BF00088830E94C4252091A3022695622F70E03D
:103C00000E949F26280F29831A828091A402843162
:103C100020F0893C18F088EC01C084E18C838B8310
:103C200097014A81698188810E944D23259623E06E
:103C3000E20EF11C82E0C13AD80709F08ECF0E9453
:103C40005A1DCDB7DEB7EBE00C94F226EF92FF924F
:103C50000F931F93CF93DF938C01C1E2D2E0E12C4D
:103C6000F12CF8018481F8E0EF16F1041CF48823AC
:103C700039F002C0811104C09E014091A40202C02B
:103C80009E0140E06091A3028091A2020E944D2318
:103C90008FEFE81AF80A239690E1E916F10409F784
:103CA0000E945A1DF801848190E001968170992745
:103CB0008483CDB7DEB7E6E00C94F726A0E0B0E051
:103CC000E4E6FEE10C94D526EC014C81042F10E0D3
:103CD0009801D8010E9470269B01AC010E943B26EE
:103CE0006B017C01E0E2F0E0E01BF10BA5E5B0E048
:103CF0009B01AC010E943B264B015C019F01DF014F
:103D00000E94C0269B01AC010E9446269B01AC018B
:103D10002C0D3D1D4E1D5F1DC501B4010E944E2698
:103D2000822FF22E99E2921728F093E0299F9001BA
:103D300011240DC025E530E0281B3109C901880F89
:103D4000991F280F391F37FF02C02F5F3F4F35954E
:103D50002795122F109591E2C92E92E0D92E00E0FE
:103D600085E5E82EEF1801FD02C08E2D01C08F2DD4
:103D70009601412F6091A3020E944D230F5F83E0C3
:103D8000C80ED11C003179F70E945A1D8C81811117
:103D900002C091E003C0803219F49FEF90931A01A2
:103DA00090911A01890F8C83CDB7DEB7ECE00C94AB
:103DB000F1260F931F93CF93DF93C1E2D2E0FE0170
:103DC000118210821282339682E0E135F807C1F742
:103DD00000E010E080911F02082E000C990B0817DC
:103DE000190794F080911901082E000C990B801787
:103DF000910754F09E014091A4026091A30280912A
:103E0000A2020E944D2303C0198218821A820F5FFA
:103E10001F4F239600311105E9F60E945A1D80912B
:103E2000180190911F02980F90931F022091190181
:103E3000280F20931901121614F49F301CF081955D
:103E400080931801DF91CF911F910F910895A0E009
:103E5000B0E0EDE2FFE10C94D926FC01828180FF05
:103E600003C0DD24DA9402C0DD24D394C1E2D2E0A1
:103E700000E010E0198218821A8294E0E92EF12CF9
